:10000000020E2A9404E50C9400223202101F900084
:10001000D8E004F07858E66001169000D3E0600262
:0700200014F02202000A3275
:03002B00020EB60C
:10003300020026BB010689828A83F0225002F7223E
:10004300BBFE01F322EF8DF0A4A8F0CF8CF0A4281F
:10005300CE8DF0A42EFE22BC000BBE0029EF8DF046
:1000630084FFADF022E4CCF875F008EF2FFFEE33F8
:10007300FEEC33FCEE9DEC984005FCEE9DFE0FD5A7
:10008300F0E9E4CEFD22EDF8F5F0EE8420D21CFE7B
:10009300ADF075F008EF2FFFED33FD4007985006E4
:1000A300D5F0F222C398FD0FD5F0EA22C2D5EC3089
:1000B300E709B2D5E4C39DFDE49CFCEE30E715B23D
:1000C300D5E4C39FFFE49EFE12005AC3E49DFDE402
:1000D3009CFC800312005A30D507C3E49FFFE49EC3
:1000E300FE22C5F0F8A3E028F0C5F0F8E5821582FA
:1000F30070021583E038F022E88FF0A4CC8BF0A4D3
:100103002CFCE98EF0A42CFC8AF0EDA42CFCEA8EE6
:10011300F0A4CDA8F08BF0A42DCC3825F0FDE98F09
:10012300F0A42CCD35F0FCEB8EF0A4FEA9F0EB8F00
:10013300F0A4CFC5F02ECD39FEE43CFCEAA42DCECD
:1001430035F0FDE43CFC2275F008758200EF2FFFCB
:10015300EE33FECD33CDCC33CCC58233C5829BED9C
:100163009AEC99E58298400CF582EE9BFEED9AFDA0
:10017300EC99FC0FD5F0D6E4CEFBE4CDFAE4CCF950
:10018300A88222B800C1B90059BA002DEC8BF084C3
:10019300CFCECDFCE5F0CBF97818EF2FFFEE33FE91
:1001A300ED33FDEC33FCEB33FB10D703994004EB49
:1001B30099FB0FD8E5E4F9FA227818EF2FFFEE3315
:1001C300FEED33FDEC33FCC933C910D7059BE99A27
:1001D3004007EC9BFCE99AF90FD8E0E4C9FAE4CCB8
:1001E300FB2275F010EF2FFFEE33FEED33FDCC3322
:1001F300CCC833C810D7079BEC9AE899400AED9B0B
:10020300FDEC9AFCE899F80FD5F0DAE4CDFBE4CCE9
:10021300FAE4C8F922E8600FECC313FCED13FDEE1A
:1002230013FEEF13FFD8F122A42582F582E5F03502
:1002330083F58322E493FB740193FA740293F92206
:10024300EC8EF0A4CCC5F0CCCDF8EFA4CEC5F02D48
:10025300FDE43CFCE8A42EC8C5F03DFDE43CFCEF06
:10026300A4FFE5F028FEE43DFDE43CFC228F358C41
:10027300368D37E4F543F544F541F542F538E53875
:10028300C39535400302035A900099E0FF65387027
:100293001CE5192FFFE412063AFCA3E0FD12062524
:1002A300FEA3E0C39DF540EE9CF53F80641206116A
:1002B3001206311206FE8F3C8E3B8D3A8C39E519BE
:1002C3002538FFE412061C120714AF3CAE3B1201A3
:1002D300868E3D8F3E120611120631120709953E96
:1002E300FFEE953DAB07FAE4F9F8AF3CAE3BAD3A10
:1002F300AC391201868E3D8F3E900099E02519FF9F
:10030300E412061CFEA3E0C3953EF540EE953DF5D1
:100313003FC3E53F648094805005E4F53FF540D347
:10032300E5409542E53F9541401485454685414367
:10033300854244853845853F418540428014D3E555
:10034300409544E53F95434009853846853F4385BD
:1003530040440538020281E5422544FFE541354327
:10036300FEC3EF9537EE953650057EFF7FFF22E5FE
:1003730036C313FEE53713FFC3E5429FF540E5415E
:100383009EF53FFEAF407C007D0A1200481206E74F
:10039300EDD3941F40027D1FEDAC36AD371206A39B
:1003A300CEC313CE13D8F9F53E8E3D2542F542E573
:1003B3003D3541F541E53E2544F544E53D3543F5FD
:1003C30043E544AE437807C333CE33CED8F9FF12A7
:1003D30006E79000F6E07002A3E070051206C08005
:1003E3000D1206F1CEC313CE13D8F91206791207F4
:1003F3001ECEC313CE13D8F9FD9000B0E545F075BA
:10040300F040A485F047F548E5451206D05002AD0B
:1004130007E54512064FC333CE33CED8F912066132
:10042300AD07AC06E545700AE53514B54604C204CC
:10043300801BE53514B54508E5467004D204800DEC
:10044300E545C395465004D2048002C20430040C2F
:10045300ED2548F548EC3547F5478022E548454703
:100463007011E53575F040A4AEF024FFF548EE3485
:10047300FFF547C3E5489DF548E5479CF547AE477B
:10048300AF4822C203751906200107D2017F041267
:1004930010607D147C007F04120270EFF47002EE92
:1004A300F46002C2029000F5E0F960030205909047
:1004B30000F4E06003020560EFF47002EEF4600BF9
:1004C3007401F09000D704F00205E0851932120A96
:1004D3008740030205E0120A68E532120A5CE0FA7B
:1004E300A3E0FBD39DEA9CE5324007120A6AC3EB03
:1004F3008014120A5CE0FCA3E0FDE532120AE4F585
:1005030083E0FAA3E0C39DF534EA9CF533D3E534E5
:100513009408E5339400502174EA2532120A7FE0EF
:100523007036120A68E532120A5CECF0A3EDF012A1
:100533000A68E532120B23800E120A68E53225E0C1
:100543002402F582E43400F583ECF0A3EDF074EAC1
:100553002532120A7F7432F005320204D1EFF470AF
:1005630002EEF4600D9000D7E070729000F504F095
:10057300806BE49000F4F0851932120A87505E74A0
:10058300EA2532120A7F7432F0053280EDE9640104
:10059300704B9000F4E06011EFF47002EEF4703DE4
:1005A300F09000D77402F08034EFF47002EEF47030
:1005B300269000D7E070269000F5F0A3F0A3120A6E
:1005C300F6851932120A87501474EA2532120A7F0B
:1005D3007432F0053280ED9000F47401F09000F570
:1005E300E064017012EFF47002EEF4600D9000D439
:1005F300EEF0A3EFF08003120AF79000D4E0F4705A
:1006030003A3E0F4600475180222E4F518229000B5
:1006130099E0AD197C002DFFEC33FEEF25E0FFEEF2
:1006230033FE74162FF58274003EF583E022FAA39D
:10063300E0FBED2538FFEC33FEEF25E0FFEE33FE64
:10064300749A2FF58274003EF583E0229013309361
:10065300FCFFEDC39FFFE49400FEEF780522FFEC5F
:10066300FDC374809DFDE49400FC0200AF75F002AD
:1006730090001602022BFFC3EB9FFFEA9E9000F649
:10068300F0A3EFF0EDFF9000F6E48FF00200E5E554
:100693000090009A75F00212022BE0FEA3E0FF2205
:1006A300FFC374209FFFE49400FE120048EF780616
:1006B30022C3EB9FEE6480F8EA64809822ED75F024
:1006C30004A4FF9000F6E5F0F0A3EFF022901330BE
:1006D30093FFEDC39F22E500C313FEE50013FFC3A1
:1006E300E5009F22AC41AD4212005AAD07229000B3
:1006F300F6E0FAA3E0FBAE02780222FEA3E0FFAD30
:1007030003AC02020243FEA3E02BFFEE3AFEC3EF6B
:1007130022FEA3E0FBAA06E4F9F8229000F6E0FE2D
:10072300A3E0780222AC00AD0012005AAD0722E428
:10073300F530F52FF52EF52DF53175E8E390803082
:10074300E04440F075A081E4F5A375A24B75A1A523
:10075300D2AF120D9D9080077402F0C2871210A1D0
:10076300E48F308E2FF52EF52DAD2EAC2D7808129B
:1007730002188F1385301485140F8513105389FCC9
:10078300758CFB758A1BD28CD2A9C2B9120FDC906F
:1007930000D4E0FEA3E0FFBEFF06BFFF03754B01DD
:1007A300EFF47002EEF4602D9000D6E070277549E7
:1007B30001F54B7531019000D4E0FEA3E02415F55B
:1007C3008274123EF583E493F54AC374EF954AF5B8
:1007D3004A2410F54A9000D6E0FF6043754901E4CE
:1007E300F54B753103EF24FE601924FE601A24FCD7
:1007F300601B24F8601C24F0601D241F701E754AC2
:1008030008801C754A0D8017754A0E8012754A04BC
:10081300800D754A068008754A028003E4F5499005
:1008230000D4E0B4FF08A3E0B4FF03754B01E5492E
:100833006401600302078FC2AFF508F549F508D2DA
:100843008CC2AF854A11D2AF02078FE50914602C21
:1008530014604814700302092F2403600302094B38
:10086300D287050DE50D7002050CC312000350037A
:1008730002094BE4F50CF50D75090122C287050D3C
:10088300E50D7002050CC39478E50C940050030247
:10089300094BE4F50CF50D75090222E512700B7591
:1008A3001201740F250AF8E6F50B050DE50D70022C
:1008B300050CE50B30E726D3E50D940CE50C94000D
:1008C3005004D2878044C3E50D940DE50C94004099
:1008D30039C287E50D6410450C702F8021D3E50DD7
:1008E3001200035004D2878021C3E50D9405E50C63
:1008F30094004016C287E50D6410450C700CF50C8E
:10090300F50DE50B25E0F50B050EE50E64087038D3
:10091300F50EF512050AE50A6403702CF50AE54B9A
:100923006401700475090322E4F50922050DE50D40
:100933007002050CD31200035003D28722C287E44E
:10094300F50CF50DF509C28C22E4F532E532120AF5
:10095300EE4003020A20120A5AE0FCA3E0FD120A49
:10096300318F33E532120A6A120A318F34EF64028F
:100973006007EF64036002C202E5337030E5347050
:100983001B120B00700E120A7BE06003020A1BEFBE
:100993004EF68000120A7B7402F0807C120B00601A
:1009A30068120A7BE07071EFF45EF68015E534702F
:1009B3000C120A48EEF0A3EFF0E4FD80567859E6F6
:1009C3006011E532120B23120A53EEF0A3EFF07D10
:1009D300028040120A5AE0FEA3E0FFE532120A6ADF
:1009E3007B1E7A0012117CEF601F120A7BE07028D5
:1009F300120A48EEF0A3EFF0E532120AE4120AA657
:100A0300E532120ACA7D02800A120A48EEF0A3EF09
:100A1300F0AD34AF32121202053202094F7859E6B3
:100A23009000D6F0600475180122E4F51822E5322F
:100A33009013349378595624FF92037B1E7A00AFA8
:100A430032120F2F22E53225E0249AF582E4340096
:100A5300F583E0FEA3E0FFE53225E02402F582E41E
:100A63003400F58322E53225E0249AF582E434004C
:100A7300F583E0FCA3E0FD2274EA2532F582E43439
:100A830000F58322E5192404FDE433FCC3E5329D1C
:100A9300EC6480F874809822E53225E024B1F58275
:100AA300E43400F583E0FEA3E0FF2274D92532F598
:100AB30082E43400F58322E53275F00AA4242AF592
:100AC30082E43400F5832225E02416F582E4340021
:100AD300F583EEF0A3EFF022E0C3940574809480D5
:100AE3002225E0249AF582E4340022C3940674801C
:100AF300948022F074FF9000D4F0A3F022E53290AA
:100B0300133493FF7859E6FEEF5E227857E624010B
:100B1300FFE433FEC32225E024B1F582E43400224E
:100B230025E02416F582E4340022900098E0701545
:100B3300C2009000D8F0F516120F8E900098740240
:100B4300F075153222900098E064026003020C08ED
:100B5300200003020C08C2001515E5156003020C02
:100B6300087858F6F532120B0EE5329FEE120A940E
:100B73004003020C04E4FFEF120ADC501CE53212BE
:100B83000B19120A73E532120ABC75F002EF120256
:100B93002BECF0A3EDF00F80DE74D92532120AB2EC
:100BA300E4F0E5327857666058120A9BE532120A80
:100BB300CA120A9BE532120A5CEEF0A3EFF0E532AB
:100BC300120AEE502DE53225E025E02416F582E4E5
:100BD3003413F583E493FE740193FFE53225E02497
:100BE300C7F582E43400120AD37D02AF3212120237
:100BF300800A74EA2532120A7F7432F00532020B3E
:100C030069784C760122908109E054E06004E04465
:100C1300E0F0E5FB30E00975FB0185E22185E12287
:100C2300E5FB30E10975FB0285E42385E324E5FB5D
:100C330030E20975FB0485E62585E526E5FB30E30F
:100C43000975FB0885D92785E728E5FB30E4097595
:100C5300FB1085DB2985DA2AE5FB30E50975FB20E6
:100C630085DD2B85DC2CE4FFEF120AEE502DEF25FA
:100C7300E02421F8E6FC08E6FDE5162F120B19F532
:100C830083ECF0A3EDF0EFFDE5162DFDE433FC78E6
:100C930057E66D7001EC60030F80CDE5162406FF67
:100CA300E433FE7857E6FDD3EF9D7480F86E9840E9
:100CB30007D200E4F516800674062516F516120F02
:100CC3008E9000D8E0600214F09000F9E0FF9000ED
:100CD300F8E0FE6F6006A3EEF075A1A522E4F532FD
:100CE300120B0EE5329FEE120A944003020D9C1282
:100CF3000AAEE004F0120AAE120ADB4005120AAE95
:100D0300E4F0C2ADE532120A9D120ABAC083C08272
:100D1300120AAEE0D082D08375F00212022BEEF0FD
:100D2300A3EFF0D2ADE4F533F534F535F53674FFC2
:100D3300F537F538E4FFEF120ADC5035120ABA75BD
:100D4300F002EF12022BE0FCA3E0FD2534F534ECB6
:100D53003533F533D3ED9536EC953540048C358D2D
:100D630036C3ED9538EC953750048C378D380F80AA
:100D7300C5C3E5349536FFE5339535FEC3EF9538A6
:100D8300FFEE9537FE7C007D0312005AE532120A0E
:100D9300E4120AD30532020CE3227857760AE4FF01
:100DA300FEEEFD7C00C3940A74809480502AC3ED48
:100DB300120AEFEE501125E025E02414F582E43405
:100DC30013F5837401800390132693FDAC070F740E
:100DD3004D2CF8A6050E80C9908030E04440F07594
:100DE300D580E4F5D6D2AD12114D75F90A75F840E8
:100DF3009081037457F0D2ADC200E49000D6F0782E
:100E030059F6F518C2019000F5F09000F4120AF6B5
:100E1300E49000F6F0A3F0784CF6900098F0900080
:100E2300F9F09000F8F022787FE4F6D8FD75815B45
:100E3300020E71020732E493A3F8E493A34003F68E
:100E43008001F208DFF48029E493A3F85407240C0B
:100E5300C8C333C4540F4420C8834004F4568001EC
:100E630046F6DFE4800B0102040810204080901155
:100E7300AAE47E019360BCA3FF543F30E509541FED
:100E8300FEE493A360010ECF54C025E060A840B8F0
:100E9300E493A3FAE493A3F8E493A3C8C582C8CA6E
:100EA300C583CAF0A3C8C582C8CAC583CADFE9DE41
:100EB300E780BEC0E0C0F0C083C082C0D075D00060
:100EC300C000C001C002C003C004C005C006C00703
:100ED300E5D530E03443D5011210DBE51D451C6038
:100EE30008E51D151D7002151C051EC3E51E948023
:100EF300748094804006751E0012000EC3E50894AA
:100F0300FA7480948050020508AFFBEF6003120C63
:100F130009D007D006D005D004D003D002D001D029
:100F230000D0D0D082D083D0F0D0E0328A358B3657
:100F3300A907E9120670E0FEA3E0C39DFFEE9CAB98
:100F430007FAE99000C712069730030B7C007D096E
:100F53001200480D1200AF1206B440037F0022D3E3
:100F6300EB9536E5351206B840037F0122C3EA64E8
:100F730080948040037F0222C3E49536FFE49535D5
:100F8300FE1206B47F0440027F0322E4FEEEC39404
:100F9300065042EEFDE5162DFDE433FC7857E6FBE3
:100FA300C3ED9B7480F86C98401AAF067D0E121146
:100FB30015EE04FCECC39406501BAF04E4FD1211C0
:100FC300150C80F0AF06E5162E244DF8E604FD124D
:100FD30011150E80B843F88022784CE6146006049D
:100FE3007039020B2D300022C2009000F9E004900A
:100FF30000F8F0120CE0D202E51864026003120953
:101003004CE518640160031204869000D8120ADBD1
:101013004009E4F5F875FB3F120D9D22C0E0C0F0D6
:10102300C083C082C0D075D000C000C001C002C060
:1010330003C004C005C006C007758CFB758A1B126C
:10104300084ED007D006D005D004D003D002D0017B
:10105300D000D0D0D082D083D0F0D0E032A90774B2
:10106300FFF535F536AF19E4FEE92519FDE433FC48
:10107300EFC39DEC6480F8748098502175F002EF03
:10108300120673E0FCA3E0FDC39536EC95355009D9
:10109300900099EEF08C358D360F0E80CC2290FCAB
:1010A300017480F0E490FC06F090FC05F090FC01E4
:1010B3007481F0A3E0FFE48F35F534F533F532AEF8
:1010C30034AD33AC321211DA1211D61211D6F53215
:1010D300E490FC01F0AC3222900000E004F0E0C3A5
:1010E3009404748094804029E4F0FF7857E6FEEF7F
:1010F300C39E501574EA2F120A7FE0600974EA2F29
:10110300120A7FE014F00F80E29000D7E06002142F
:10111300F022EF14601614601914601C14601F147D
:10112300602224057023ED4440F5FC22ED4440F594
:10113300FD22ED4440F5FE22ED4440F5FF22ED444F
:1011430040F5F122ED4440F5F22290801D7404F045
:10115300E4FF7857E6FEEFC39E501D744D2FF8E66B
:1011630075F003A4243FF582E43413F583120237A8
:1011730074041200360F80DA22C3EF9DFFEE9CFE4B
:10118300D3EF9BEA6480F8EE6480985017C3E49B26
:10119300FDE49AFCC3EF9DEC6480F8EE6480984014
:1011A300037F01227F0022014900014A00014B0015
:1011B300011E00010900020C0000030F00000001E2
:1011C3000A00010E00010B000112004100000001A2
:1011D300150000F532FCE4FB7A01F9F81200FB8FED
:1011E300358E348D338C3290FC02E0FFE5354FFFB2
:1011F300E534FEE533FDE5328F358E348D3322ED54
:1012030090133A93FE74EA2FF582E43400F583EEEB
:10121300F022000102030405060708090A0B0C0D5E
:10122300101010111212131415161718191A1B1C6B
:101233001D1E1F20212223242525262728292A2B6A
:101243002C2D2E2F30313233343536373838393A66
:101253003B3C3D3E3F404142434445464748494A63
:101263004A4B4C4D4E4F5051525354555657585963
:101273005A5B5C5D5D5E5F6061626364656667685F
:10128300696A6B6C6D6E6F7070717273747576775B
:1012930078797A7B7C7D7E7F808182828384858658
:1012A3008788898A8B8C8D8E8F9091929394959554
:1012B300969798999A9B9C9D9E9FA0A1A2A3A4A553
:1012C300A6A7A8A8A9AAABACADAEAFB0B1B2B3B450
:1012D300B5B6B7B8B9BABABBBCBDBEBFC0C1C2C34D
:1012E300C4C5C6C7C8C9CACBCCCDCDCECFD0D1D249
:1012F300D3D4D5D6D7D8D9DADBDCDDDEDFE0E0E145
:10130300E2E3E4E5E6E7E8E9EAEBECEDEEEFEF0034
:1013130000000400320005003200070050000900FD
:1013230032000A0032000C00320B0306081B0A15B8
:101333001E0102040810200264501E1E01801901C0
:101343008018018007018006018005018004018067
:101353000301800201800101800001801C01801BC8
:0313630001801AEC
:00000001FF
